:020000040000FA
:10000000B0220020150200001D0200001F020000A7
:100010002102000023020000250200000000000071
:1000200000000000000000000000000027020000A7
:1000300029020000000000002B0200002D02000039
:100040002F0200002F0200009D0500002F0200007B
:100050002F0200002F0200002F0200002F020000DC
:100060002F0200002F0200002F0200002F020000CC
:100070002F0200002F0200002F0200002F020000BC
:100080002F0200002F0200002F0200002F020000AC
:100090002F0200002F0200002F0200002F0200009C
:1000A0002F0200002F0200002F0200002F0200008C
:1000B0002F0200002F0200000000000000000000DE
:1000C0002F0200002F0200002F0200002F0200006C
:1000D0002F0200002F0200002F020000000000008D
:1000E0000000000000000000000000000000000010
:1000F0000000000000000000000000000000000000
:1001000000000000000000000000000000000000EF
:1001100000000000000000000000000000000000DF
:1001200000000000000000000000000000000000CF
:1001300000000000000000000000000000000000BF
:1001400000000000000000000000000000000000AF
:10015000000000000000000000000000000000009F
:10016000000000000000000000000000000000008F
:10017000000000000000000000000000000000007F
:10018000000000000000000000000000000000006F
:10019000000000000000000000000000000000005F
:1001A000000000000000000000000000000000004F
:1001B000000000000000000000000000000000003F
:1001C000000000000000000000000000000000002F
:1001D000000000000000000000000000000000001F
:1001E000000000000000000000000000000000000F
:1001F00000000000000000000000000000000000FF
:10020000DFF80CD000F02AF800480047250A00006B
:10021000B02200200648804706480047FEE7FEE778
:10022000FEE7FEE7FEE7FEE7FEE7FEE7FEE7FEE7A6
:10023000810200000102000040EA01039B0703D095
:1002400009E008C9121F08C0042AFAD203E011F815
:10025000013B00F8013B521EF9D27047064C074D96
:1002600006E0E06840F0010394E807009847103486
:10027000AC42F6D3FFF7C8FFB8150000D815000050
:10028000F0B5B5480023021D0178101D01254FF07F
:10029000805406290BD11678360708D10678C6F3A4
:1002A0000316032E06D0042E04D0052E02D00629F4
:1002B00007D00EE0B4F82463A84FC6F304263E60CE
:1002C00002E01678360704D10678C6F30316032E2B
:1002D00002D0062904D00FE0A24FA14E7E670EE0A7
:1002E0001678360708D10678C6F30316032E06D013
:1002F000042E04D0052E02D0062907D00EE0D4F833
:100300004462994FC6F342363E6002E016783607E3
:1003100004D10678C6F30316032E02D0062906D0B0
:1003200011E0924E376827F0807737600EE016783C
:10033000360708D10678C6F30316032E06D0042E1E
:1003400004D0052E02D006290AD011E04FF08046D5
:10035000C6F80C31C6F81031834E361F336002E008
:100360001678360704D10678C6F30316032E02D09A
:10037000062905D00CE07C4F032664373E600AE076
:100380001678360704D10678C6F30316032E02D07A
:1003900006290DD014E0764F05263E60744E78365F
:1003A0003560734E083633603F263F1D3E6002E0E5
:1003B0001678360704D10678C6F30316052E02D048
:1003C000062957D062E06B4E36686B4F3E60694E2F
:1003D000361D36683F1D3E60664E083636683F1D46
:1003E0003E60644E0C3636683F1D3E60614E1036EE
:1003F00036683F1D3E605F4E143636683F1D3E60D6
:100400005C4E183636685C4F20373E60594E1C36BD
:1004100036683F1D3E60574E203636683F1D3E60B1
:10042000544E243636683F1D3E60524E283636689C
:100430003F1D3E604F4E2C3636683F1D3E604D4E90
:10044000303636684C4F40373E604A4E3436366858
:100450003F1D3E60474E383636683F1D3E60454E74
:100460003C3636683F1D3E60424E403636683F1D82
:100470003E6002E01678360708D10678C6F3031608
:10048000032E06D0042E04D0052E02D0062907D054
:1004900019E0D4F85812394A01F04F01116002E016
:1004A000117809070FD10078C0F30310032803D097
:1004B000042801D0052806D131480168C90702D0B7
:1004C0006FF001010160D4F83001062808D1D4F89A
:1004D0003401062804D12B48016841F48061016091
:1004E00022487438016841F470010160BFF34F8FF6
:1004F000BFF36F8F4FF01021D1F80002002803DB0B
:10050000D1F80402002822DA1F4A15601F48046847
:10051000002CFCD01524C1F800420568002DFCD049
:10052000C1F8044201680029FCD013600168002969
:10053000FCD0BFF34F8F0D48F0380168144A01F426
:10054000E06111430160BFF34F8F00BFFDE7124927
:1005500010480860F0BD0000E00F00F04035014099
:100560000DF0ADBA00C007403C050040FCED00E0D6
:10057000105600400404001020C50040E40E004066
:10058000000400403C17004004E5014000E4014045
:100590000400FA050090D0033800002001480068EC
:1005A000004700000C000020014A024900F013B887
:1005B000950900003400002002E008C8121F08C19D
:1005C000002AFAD170477047002001E001C1121FD4
:1005D000002AFBD170472DE9F04116460F4604462C
:1005E000002503E03946B047641C6D1C20780028C4
:1005F000F8D12846BDE8F08172B609480068C00706
:1006000000D000BEBFF34F8F0548E4380168054AAB
:1006100001F4E06111430160BFF34F8F00BFFDE7BC
:10062000F0ED00E00400FA050EB500210091CDE9DF
:1006300001106A4644F20100FFF7DEFF0EBD10B55F
:100640008268C368934203D000F091F9002010BD86
:10065000052010BD29B112B1531E134203D0092049
:1006600070470E2070470160838000218160C16067
:100670000846704710B58268C3689A1A83889A4200
:1006800003D800F07EF9002010BD042010BD00004A
:1006900070B50A4E01460A48B578FFF7D0FF044608
:1006A0004DB10020B070711C0122C81D00F03CFA51
:1006B00008B1FFF7B9FF204670BD0000140000200C
:1006C0008C020020F0B5244E89B01F460D00044670
:1006D00072603FD0A888296882B22048FFF7BAFF2D
:1006E000002835D1A889A96882B21C481030FFF7CC
:1006F000B1FF00282CD1202219496846FFF79CFD44
:1007000060690690207C00B101208DF814008DF8FE
:100710001C70607C00B10E208DF81500E06802901E
:10072000A068039020680190606800900A480D4A14
:100730006946083000F0C4F9002809D1B07020687B
:10074000401C05D004490122491CC81D00F0ECF9E9
:1007500009B0F0BD0720FBE7140000208C02002048
:10076000981500005512000010B501461048FFF71B
:1007700081FF040019D10F480F4A0178515C19B16B
:10078000001D00F0E7FC02E00C3000F0CBFB60B98C
:10079000084907480839FFF752FF30B905490122D7
:1007A0000839044800F0D0F90446204610BD000086
:1007B0009C0200201C0000200000002000F002B875
:1007C00000F008B872B602480168491C0160704721
:1007D0003000002003490868401E086000D162B65E
:1007E00070470000300000202DE9F04106460868FF
:1007F0000C46411C4FF0A0474FF0010506D005FA0A
:1008000000F1C7F80815206800F0F6F96068411C8F
:1008100002D0002100F0DEF93168A069C1F824059A
:10082000607D227D31681043C1F86C05D4E9001267
:100830003068C0F81425C0F80C15207D012815D1AA
:10084000A068411C02D0002100F0C4F9E068411CFE
:1008500005D08540C7F80855E06800F0CDF9D4E927
:1008600002123068C0F80825C0F81015BDE8F08104
:100870002DE9F041064608680C46411C4FF0A047A0
:100880004FF0010506D005FA00F1C7F808152068F9
:1008900000F0BCF96068411C02D0002100F0A3F90F
:1008A0003168A069C1F82405607D217D3268084364
:1008B000C2F86C05D4E900123068C0F80C15C0F815
:1008C0001425207D012815D1A068411C02D00021EB
:1008D00000F089F9E068411C05D08540C7F808554B
:1008E000E06800F093F9D4E902123068C0F80825F6
:1008F000C0F81015BDE8F0812DE9FC410646C0079F
:100900004FF000050ED0104F00240122385D0095F5
:1009100000231146019500F027F9641C042CF4D340
:1009200000F01CF8B0070DD5074E0024361D00223C
:10093000305D032300951146019500F015F9641C04
:10094000042CF4D3BDE8FC81881500000249085C42
:10095000012100F065B900008815000010B50024E1
:100960002046FFF7F3FF641C042CF9D310BD826806
:1009700083881A4003689A5C0A708168491C816008
:100980007047C26883881A4003689954C168491C3B
:10099000C160704710B50446C0B2FFF7E5FE2046BF
:1009A00010BD000070B50D46044600684FF4887114
:1009B00000F057F94FF49071206800F052F94FF4AD
:1009C0009271206800F04DF94FF4A271206800F098
:1009D00048F920681249C0F8041320686907000B21
:1009E00040B2090E002806DA00F00F0000F1E02006
:1009F00080F8141D03E000F1E02080F80014206866
:100A00000121000B40B200F01F029140400980001C
:100A100000F1E020C0F88012C0F8001170BD0000A5
:100A2000100302008AB00120FFF766FF1822164962
:100A30006846FFF701FC1548069015494FF4807091
:100A4000CDE9070109900723124A06A96846FFF776
:100A500039FE08B1FFF7E8FD0FA0FFF7A5FD06A8D6
:100A6000FFF716FE0028FAD19DF81800FFF77CFE6C
:100A70000028F9D19DF81800712801D05128EED135
:100A80000CA0FFF791FDFEE7701500003C00002070
:100A90003C010020431200000D0A554152542065CC
:100AA00078616D706C6520737461727465642E0D6D
:100AB0000A000000200D0A45786974210D0A000023
:100AC000F0B505460478154889B0164640F824204C
:100AD000124A0869121DA2F1080742F82400487F53
:100AE000385520226846FFF7A7FB04942878385C25
:100AF00048B10EB10A4A00E000226946281D00F004
:100B000029FA09B0F0BD0EB1064A00E0002269469C
:100B100005F10C0000F0D4F8F3E700000400002019
:100B20004D140000F512000030B40378054CE35C6E
:100B30001BB130BC001D00F043BA30BC0C3000F0DB
:100B400029B900000000002030B40378054CE35CB4
:100B50001BB130BC001D00F0B5BA30BC0C3000F049
:100B60008FB900000000002070B541EA4201DDE9C4
:100B700004564FF0A04441EA830141EA052104EB09
:100B8000800041EA0641C0F8001770BD70B541EA27
:100B90004201DDE904564FF0A04441EA830141EAF5
:100BA000052104EB800041EA0641C0F8001770BD42
:100BB00070B541EA4201DDE904564FF0A04441EA34
:100BC000830141EA052104EB800041EA0641C0F8B7
:100BD000001770BD1CB500220B4600921146019211
:100BE000FFF7D4FF1CBD1CB500220B460092114636
:100BF0000192FFF7DDFF1CBD1CB5002100910B46E3
:100C0000012201911146FFF7C1FF1CBD1CB5002157
:100C100000910B46012201911146FFF7C9FF1CBD4F
:100C200001224FF0A043824011B1C3F8082570475C
:100C3000C3F80C2570474058002800D001207047A9
:100C400008B5002242504058009008BDD0F8040377
:100C5000084000D0012070474058002800D00120F3
:100C6000704708B5002242504058009008BD01214D
:100C7000B1EB507F01D1012070470020704770B563
:100C80000D4600F075FA04000FD00020FFF796FD26
:100C9000207920B10020FFF793FD112070BD0120C5
:100CA000256020710020FFF78BFD002070BD000043
:100CB0000149024800F036BB3C0200200020004001
:100CC0002DE9F0410546007916460F4600EB40013C
:100CD0002D4A01EBC00102EB810494F82A1011B1F6
:100CE0000820BDE8F081294951F820102868FFF755
:100CF000C6FF08B11120F4E739462846FFF774FD16
:100D000066603869206030004FF001062FD03F7FC9
:100D10004FF48E712868FFF793FF4FF4A271286893
:100D2000FFF78EFF28681A49C0F8041328684FEAB5
:100D30004711000B40B2002806DA00F00F0000F166
:100D4000E02080F8141D03E000F1E02080F800149A
:100D50002868000B40B200F01F0206FA02F14009B9
:100D6000800000F1E020C0F88012C0F8001128686F
:100D70000421C0F800150020A061E06184F829007A
:100D800044F8140FA675ACE73C0200209015000053
:100D9000800002002DE9F05F054600794FF40176EE
:100DA00000EB400303EBC000344B03EB8004002056
:100DB000636813B12B68C3F80863A3694FF0000997
:100DC0006BB1E06938B1606810B12868C0F804639D
:100DD0001120BDE8F09FE2610120216105E0C4F827
:100DE0002490A261E160C4F81C9094F8291001439A
:100DF00002D1284600F0F8F960680028286803D07E
:100E0000C0F804630020E4E74FF4A2763146FFF710
:100E100017FFB2464FF4927B59462868FFF70BFF45
:100E200006464FF484712868FFF705FF8046514657
:100E30002868FFF700FF074648EA07003043EBD079
:100E400056EA070007D12146286800F09DF9A169FC
:100E5000606A8142E0D8C4F818900EB10320B8E768
:100E60000FB10F20B5E794F8291001200029296857
:100E700001D00860C6E74860C4E700003C020020DB
:100E80002DE9F047054600790B4600EB400101EBE8
:100E9000C000234901EB8004284600F043F810B15C
:100EA0001120BDE8F0874FF00008C4F82080A3604F
:100EB000626184F828804FF48E7647463146286870
:100EC000FFF7BEFE28684FF00109C0F808902146E0
:100ED000286800F099F9606800BBD5F800A00EE022
:100EE00094F8280008B10F2716E031465046FFF766
:100EF000A2FE0028F4D02146504600F085F9216A70
:100F000060698142F1D331462868FFF794FE0028DA
:100F1000F9D02868C0F80C90C4F814803846C0E7AF
:100F20003C020020007900EB400101EBC0000449C5
:100F300001EB80004069002800D0012070470000CC
:100F40003C0200200149024800F098BA68020020E3
:100F5000002000402DE9F0410546164600790F4675
:100F6000154A00EBC00102EB810494F8201011B186
:100F70000820BDE8F081114951F820102868FFF7DA
:100F80007EFE08B11120F4E739462846FFF770FCD1
:100F90006660386920601EB1397F2846FFF702FD80
:100FA00028680821C0F800150020A061E061012137
:100FB000606184F82010DCE76802002094150000CE
:100FC0002DE9F05F044600790E4600EBC001DFF822
:100FD000F0A017460AEB81053046FFF748FEB0B196
:100FE00068684FF000084FF4047910B12168C1F827
:100FF0000893A8694FF0000B80B1E86948B16868B0
:1010000010B12068C0F804931120BDE8F09F1020B3
:10101000FBE7EF614FF001082E6102E0EE60C5E9E9
:10102000067B00254FF488712068FFF71AFE4FF405
:10103000A2712068FFF715FE2068C0F83465C0F87B
:1010400038752068B8F1000F12D0D0F8001241F0C6
:101050002001C0F800122079D04600EBC0010AEB55
:101060008100406838B12068C0F804932846CCE776
:1010700001210160EFE74FF4887A4FF4A2795146DD
:101080002068FFF7E9FD074649462068FFF7E4FDC1
:1010900006464FF492712068FFF7DEFD014647EAED
:1010A00006000843EBD0227902EBC20308EB83026F
:1010B000C2F818B001B10325002ED7D00F25D5E70F
:1010C000680200202DE9F04704460E4600792049C9
:1010D00000EBC00001EB800517463046FFF7C7FD67
:1010E00030B1204600F036F820B11120BDE8F0877D
:1010F0001020FBE76F61AE604FF490760027314619
:101100002068FFF7AEFD4FF4AC7841462068FFF74A
:10111000A8FD2068AA686969C0F84425C0F8481588
:10112000206801218160686878B9B1464946206825
:10113000FFF792FD064641462068FFF78DFD064306
:10114000F4D000B10F27002068613846CEE70000D8
:10115000680200200079054900EBC00001EB800027
:101160004069002800D0012070470000680200207C
:101170000349884201D103487047002070470000AE
:10118000002000400C00002070B5054688690C4620
:1011900000284FF4847128460AD0FFF751FDD5F896
:1011A0001805626AE1688854606A401C606270BD1C
:1011B000FFF746FDD5F8180570BD1FB501238DF862
:1011C0000030CDE90121D0E90012684690471FBDEB
:1011D0001FB501238DF800308DF808100192D0E979
:1011E0000012684690471FBD10B5044600684FF4D2
:1011F0009271FFF725FD4FF484712068FFF720FD01
:1012000020680121016010BD70B50C4605464FF401
:101210008E71FFF715FD216AA068415C206A401CB1
:101220002062C5F81C1570BD1FB500228DF8002086
:101230000291816801914261D0E9001268469047AD
:101240001FBD0178022901D0012902D14068FFF7B2
:10125000EBB970477CB50178244D81B301290BD0DF
:1012600002292BD18DF80010C068691C0190012261
:10127000C81DFFF759FC2EE0406801781C48FFF7B5
:10128000F9F91B4C012618B18DF80060019006E0B9
:10129000A068E168814205D000208DF800006968EF
:1012A00068468847A068E168081AA188884207D87C
:1012B0000E490122491CC81DFFF736FC7CBD01E028
:1012C000AE70FBE70A4809491030FFF7B8F930B1B2
:1012D00003208DF80000696868468847EEE70349F7
:1012E000012201F10800FFF72FFCE7E714000020BE
:1012F0008C0200201FB50A4601788DF80010416865
:101300000191017A8DF80810C0680390044850F8E4
:101310002210001F50F82220684690471FBD000091
:10132000080000202DE9FF470C4605464FF40071E8
:10133000FFF78CFC01274FF40178002618B34FF417
:10134000927949462846FFF776FCE0B1494628469F
:10135000FFF776FCC5F8088394F8290000B96F60A0
:1013600002208DF80000D5F88004C5F880040390B1
:10137000A0690290E0680190A661E661D4E90012DC
:101380006846904728E004212846FFF75FFC18B321
:101390004FF484712846FFF74EFCE8B121462846F9
:1013A000FFF7F2FE616AA069884215D1E06938B1A1
:1013B000E268616AA0612069E6616662E06008E057
:1013C00094F8290000B96F60C5F80883A661E26847
:1013D000616A2046FFF7F1FE4FF48E7841462846B9
:1013E000FFF729FC78B1206A6169884202D294F83B
:1013F000280020B341462846FFF722FC616911B15D
:101400002046FFF711FF4FF4A27841462846FFF728
:1014100012FC002818D041462846FFF711FC94F82A
:10142000290000B12F60A06900280DD0A661E268F4
:10143000616A04B02046BDE8F047FFF7BEBE214612
:101440002846FFF7E1FEDEE7BDE8FF871FB50A4645
:1014500001788DF8001041680191017A8DF808102B
:10146000C0680390044850F82210001F50F8222052
:10147000684690471FBD0000080000202DE9FF418D
:101480000C464FF4927705463946FFF7E5FB0026F8
:10149000C0B139462846FFF7E4FB02208DF8000072
:1014A000D5F88004C5F880040390D5F83C058DF884
:1014B0000800E0680190A661E661D4E90012684680
:1014C000904723E04FF4887739462846FFF7C4FB5E
:1014D000E0B139462846FFF7C4FBD5F83C15A069B2
:1014E000884213D1E06960B1E268D5F8000220F0CB
:1014F0002000C5F80002E069A0612069E661E060B3
:1015000001E0A661E2682046FFF762FE4FF4A27791
:1015100039462846FFF7A0FB60B139462846FFF759
:10152000A0FBA06930B1A661D5F83C152046E26861
:10153000FFF74EFE4FF4907739462846FFF78CFBB5
:10154000002813D039462846FFF78BFB6069002836
:101550000CD0D5F84C058DF800608DF80800A06817
:1015600001906661D4E9001268469047BDE8FF81AA
:101570000800000006000000050000000700000051
:101580000000000000E0D701111213140D0E0F101F
:10159000B10C0000450F0000FFFFFFFFFFFFFFFF42
:1015A000FFFFFFFFFFFFFFFF000000000000000043
:1015B0000000D60107010000D8150000000000203F
:1015C0003C000000B8050000141600003C0000209C
:1015D00074220000C80500000000000000000000A8
:1015E00000000000000000000000000000000000FB
:1015F000000000000000000000200040000000008B
:10160000002000400000000000000000000000007A
:041610000090D00373
:0400000500000201F4
:00000001FF
